:100000000C942A000C9434000C9434000C943400AA
:100010000C9434000C9434000C9434000C94340090
:100020000C9434000C9434000C9434000C94340080
:100030000C9434000C9434000C9434000C94340070
:100040000C9434000C9434000C9434000C94400054
:100050000C94340011241FBECFE5D4E0DEBFCDBF29
:100060000E9436000C9452000C9400008FEF81BB6C
:100070008DE083BF8DE78CBF82E089BF7894FFCF8E
:100080001F920F920FB60F9211248F939F9382B3FA
:1000900091E0892782BB9F918F910F900FBE0F90A7
:0800A0001F901895F894FFCFA2
:00000001FF
